** EXPERIMENTAL (HLL) ** Open Watcom Linker Version 1.6beta1 Limited Availability
Portions Copyright (c) 1985-2002 Sybase, Inc. All Rights Reserved.
Created on:       12/01/07 19:00:26
Warning! W1121: file U:/tmp\ldconv_module_obj_de0c4f0802a11d4670.obj(U:\DEV\python-2.7.2\Modules\_sqlite\module.c): '_init_sqlite3' has already been exported
Executable Image: build/lib.os2knix-2.7/_sqlite3.pyd
creating an OS/2 EMX dynamic link library


                        +------------+
                        |   Groups   |
                        +------------+

Group                           Address              Size
=====                           =======              ====

CGROUP                          0001:00000000        00073560
DGROUP                          0002:00000000        00001ff0



                        +--------------+
                        |   Segments   |
                        +--------------+

Segment                Class          Group          Address         Size
=======                =====          =====          =======         ====

TEXT32                 CODE           CGROUP         0001:00000000   00073560
________TEXT           CODE           CGROUP         0001:00073560   00000000
DATA32                 DATA           DGROUP         0002:00000000   00001a38
SET1__os2dll           DATA           DGROUP         0002:00001a38   00000004
SET2__os2dll           DATA           DGROUP         0002:00001a3c   00000000
SET3__os2dll           DATA           DGROUP         0002:00001a3c   00000004
SET1___CTOR_LIST__     DATA           DGROUP         0002:00001a40   00000004
SET2___CTOR_LIST__     DATA           DGROUP         0002:00001a44   00000000
SET3___CTOR_LIST__     DATA           DGROUP         0002:00001a44   00000004
SET1___DTOR_LIST__     DATA           DGROUP         0002:00001a48   00000004
SET2___DTOR_LIST__     DATA           DGROUP         0002:00001a4c   00000000
SET3___DTOR_LIST__     DATA           DGROUP         0002:00001a4c   00000004
SET1___crtinit1__      DATA           DGROUP         0002:00001a50   00000004
SET2___crtinit1__      DATA           DGROUP         0002:00001a54   00000000
SET3___crtinit1__      DATA           DGROUP         0002:00001a54   00000004
SET1___crtexit1__      DATA           DGROUP         0002:00001a58   00000004
SET2___crtexit1__      DATA           DGROUP         0002:00001a5c   00000000
SET3___crtexit1__      DATA           DGROUP         0002:00001a5c   00000004
SET1___eh_frame__      DATA           DGROUP         0002:00001a60   00000004
SET2___eh_frame__      DATA           DGROUP         0002:00001a64   00000018
SET3___eh_frame__      DATA           DGROUP         0002:00001a7c   00000004
SET1___eh_init__       DATA           DGROUP         0002:00001a80   00000004
SET2___eh_init__       DATA           DGROUP         0002:00001a84   00000004
SET3___eh_init__       DATA           DGROUP         0002:00001a88   00000004
SET1___eh_term__       DATA           DGROUP         0002:00001a8c   00000004
SET2___eh_term__       DATA           DGROUP         0002:00001a90   00000004
SET3___eh_term__       DATA           DGROUP         0002:00001a94   00000004
SET1___fork_parent1__  DATA           DGROUP         0002:00001a98   00000004
SET2___fork_parent1__  DATA           DGROUP         0002:00001a9c   00000000
SET3___fork_parent1__  DATA           DGROUP         0002:00001a9c   00000004
SET1___fork_child1__   DATA           DGROUP         0002:00001aa0   00000004
SET2___fork_child1__   DATA           DGROUP         0002:00001aa4   00000000
SET3___fork_child1__   DATA           DGROUP         0002:00001aa4   00000004
________DATA           DATA           DGROUP         0002:00001ab0   00000000
BSS32                  BSS            DGROUP         0002:00001ab0   00000450
c_common               BSS            DGROUP         0002:00001f00   000000f0
________BSS            BSS            DGROUP         0002:00001ff0   00000000


                        +----------------+
                        |   Memory Map   |
                        +----------------+

* = unreferenced symbol
+ = symbol only referenced locally

Address        Symbol
=======        ======

Module: U:\usr\lib\dll0hi.obj({standard input})
0001:00000000* __text
0002:00000000* __data
0002:00000000* ___data_start
0002:00001ab0* ___bss_start
0002:00001a38+ __os2dll
0002:00001a40  ___CTOR_LIST__
0002:00001a48  ___DTOR_LIST__
0002:00001a50* ___crtinit1__
0002:00001a58* ___crtexit1__
0002:00001a60  ___eh_frame__
0002:00001a80  ___eh_init__
0002:00001a8c  ___eh_term__
0002:00001a98+ ___fork_parent1__
0002:00001aa0+ ___fork_child1__
Module: U:/tmp\ldconv_cache_obj_de0c4f0802a11bfe50.obj(U:\DEV\python-2.7.2\Modules\_sqlite\cache.c)
0001:000000a0* _pysqlite_new_node
0001:000000e8* _pysqlite_node_dealloc
0001:0000013b* _pysqlite_cache_dealloc
0001:000001e5  _pysqlite_cache_setup_types
0001:00000230* _pysqlite_cache_display
0001:000003eb  _pysqlite_cache_get
0001:00000596* _pysqlite_cache_init
0002:00000050* _pysqlite_NodeType
0002:00000120  _pysqlite_CacheType
Module: U:/tmp\ldconv_connection_obj_de0c4f0802a11c4c70.obj(U:\DEV\python-2.7.2\Modules\_sqlite\connection.c)
0001:000007c5  _pysqlite_check_connection
0001:00000a5c  _pysqlite_connection_setup_types
0001:00000a8f* _pysqlite_connection_executescript
0001:00000b5e* _pysqlite_connection_executemany
0001:00000c2a* _pysqlite_connection_execute
0001:00000ce9  _pysqlite_connection_register_cursor
0001:00000df2  _pysqlite_check_thread
0001:00000e4a* _pysqlite_connection_cursor
0001:00000fde* __pysqlite_build_py_params
0001:000013dd* __pysqlite_set_result
0001:000015a8* __pysqlite_final_callback
0001:000016b7* __pysqlite_func_callback
0001:000017a7  __pysqlite_connection_begin
0001:0000189e* _pysqlite_connection_dealloc
0001:00001a8b* _pysqlite_do_all_statements
0001:00001b71* _pysqlite_flush_statement_cache
0001:00001e2e  _pysqlite_connection_commit
0001:00002143* _pysqlite_connection_init
0001:00002565* _pysqlite_connection_close
0001:000026d9* _pysqlite_connection_create_aggregate
0001:0000282b* _pysqlite_connection_create_function
0001:00002968* _pysqlite_connection_rollback
0001:00002d79* _pysqlite_connection_call
0002:00000220  _pysqlite_ConnectionType
Module: U:/tmp\ldconv_cursor_obj_de0c4f0802a11ca648.obj(U:\DEV\python-2.7.2\Modules\_sqlite\cursor.c)
0001:00003740* _pysqlite_cursor_getiter
0001:0000374b* _pysqlite_noop
0001:00003988  _pysqlite_cursor_setup_types
0001:000039a6* _pysqlite_cursor_close
0001:00003a93* _pysqlite_cursor_executescript
0001:00003cc9* __pysqlite_build_column_name
0001:00003d42* _pysqlite_unicode_from_string
0001:00003df3* __pysqlite_fetch_one_row
0001:00004262* __pysqlite_get_converter
0001:000042c3* _pysqlite_build_row_cast_map
0001:00004590* _pysqlite_cursor_iternext
0001:00004738* _pysqlite_cursor_fetchall
0001:000047d6* _pysqlite_cursor_fetchmany
0001:0000489d* _pysqlite_cursor_fetchone
0001:000049b3* __pysqlite_query_execute
0001:00005599* _pysqlite_cursor_executemany
0001:000055bb* _pysqlite_cursor_execute
0002:000005f0  _pysqlite_CursorType
Module: U:/tmp\ldconv_microprotocols_obj_de0c4f0802a11d0bd8.obj(U:\DEV\python-2.7.2\Modules\_sqlite\microprotocols.c)
0002:00001f00+ _psyco_adapters
0001:00005859  _pysqlite_microprotocols_adapt
0001:000059f8  _pysqlite_adapt
0001:00005a59  _pysqlite_microprotocols_add
0001:00005ad7  _pysqlite_microprotocols_init
Module: U:/tmp\ldconv_module_obj_de0c4f0802a11d4670.obj(U:\DEV\python-2.7.2\Modules\_sqlite\module.c)
0002:00001f10  __enable_callback_tracebacks
0002:00001f20  _converters
0002:00001f30  _pysqlite_BaseTypeAdapted
0002:00001f40  _pysqlite_OperationalError
0002:00001f50  _pysqlite_Error
0002:00001f60  _pysqlite_Warning
0002:00001f70  _pysqlite_InterfaceError
0002:00001f80  _pysqlite_DatabaseError
0002:00001f90  _pysqlite_InternalError
0002:00001fa0  _pysqlite_ProgrammingError
0002:00001fb0  _pysqlite_IntegrityError
0002:00001fc0  _pysqlite_DataError
0002:00001fd0  _pysqlite_NotSupportedError
0002:00001fe0  _pysqlite_OptimizedUnicode
0001:0000601f  _init_sqlite3
Module: U:/tmp\ldconv_prepare_protocol_obj_de0c4f0802a11d9490.obj(U:\DEV\python-2.7.2\Modules\_sqlite\prepare_protocol.c)
0001:00006a10* _pysqlite_prepare_protocol_init
0001:00006a17* _pysqlite_prepare_protocol_dealloc
0001:00006a2c  _pysqlite_prepare_protocol_setup_types
0002:00000bf0  _pysqlite_PrepareProtocolType
Module: U:/tmp\ldconv_row_obj_de0c4f0802a11de698.obj(U:\DEV\python-2.7.2\Modules\_sqlite\row.c)
0001:00006a70* _pysqlite_row_dealloc
0001:00006acb* _pysqlite_row_length
0001:00006bd4  _pysqlite_row_setup_types
0001:00006bfc* _pysqlite_row_keys
0001:00006cc4* _pysqlite_row_subscript
0001:00006e77* _pysqlite_row_init
0002:00000cd0  _pysqlite_RowType
0002:00000cc0* _pysqlite_row_as_mapping
Module: U:/tmp\ldconv_statement_obj_de0c4f0802a11e2ce8.obj(U:\DEV\python-2.7.2\Modules\_sqlite\statement.c)
0001:00006f70  _pysqlite_statement_mark_dirty
0001:00006f7f  _pysqlite_statement_setup_types
0001:00006f9d  _pysqlite_statement_finalize
0001:00006fe6* _pysqlite_statement_dealloc
0001:0000705c  _pysqlite_statement_reset
0001:000070b0  _pysqlite_statement_recompile
0001:00007149  _pysqlite_statement_create
0001:00007495* _pysqlite_statement_bind_parameter
0001:0000785b  _pysqlite_statement_bind_parameters
0002:00000dc0  _pysqlite_StatementType
Module: U:/tmp\ldconv_util_obj_de0c4f0802a11e7720.obj(U:\DEV\python-2.7.2\Modules\_sqlite\util.c)
0001:00007ce0  __pysqlite_seterror
0001:00007e52  _pysqlite_step
Module: U:\usr\local446\lib\libc_dll.lib(dllinit.obj)
0001:00007e90  _DLL_InitTerm
Module: U:\usr\lib\libend.lib(src/libend/386/endlink386.asm)
0002:00001ff0  _end
0002:00001ab0  _edata
Module: U:\usr\lib\libend.lib(src/libend/386/end.asm)
0001:00073560* _etext
0001:00073560* __etext
0000:00000000* WEAK$ZERO
0002:00001ff0  __end
0002:00001ab0  __edata
Module: U:\extras\lib\sqlite3.lib(sqlite3.obj)
0001:00007ef0* _sqlite3_status
0001:00007f2f* _sqlite3_db_status
0001:000083e1* _sqlite3_mutex_free
0001:000083f8* _sqlite3_mutex_enter
0001:0000840f* _sqlite3_mutex_try
0001:00008429* _sqlite3_mutex_leave
0001:00008440* _sqlite3_vfs_unregister
0001:000084b8* _sqlite3_release_memory
0001:000084bf* _sqlite3_memory_used
0001:000084ca* _sqlite3_memory_highwater
0001:0000853b* _sqlite3_memory_alarm
0001:00008731* _sqlite3_free
0001:00008b72* _sqlite3_strnicmp
0001:0000aa21  _sqlite3_enable_shared_cache
0001:0000b18c* _sqlite3_backup_remaining
0001:0000b197* _sqlite3_backup_pagecount
0001:0000b1a2* _sqlite3_sql
0001:0000b78e* _sqlite3_expired
0001:0000b7a8  _sqlite3_value_type
0001:0000b7b4  _sqlite3_user_data
0001:0000b7c1* _sqlite3_context_db_handle
0001:0000b7cc* _sqlite3_get_auxdata
0001:0000b7f1* _sqlite3_aggregate_count
0001:0000b7ff  _sqlite3_column_count
0001:0000b811  _sqlite3_data_count
0001:0000b8a4  _sqlite3_column_name
0001:0000b8c2* _sqlite3_column_name16
0001:0000b8e0  _sqlite3_column_decltype
0001:0000b8fe* _sqlite3_column_decltype16
0001:0000b91c  _sqlite3_bind_parameter_count
0001:0000b9ab  _sqlite3_bind_parameter_name
0001:0000b9dc* _sqlite3_db_handle
0001:0000b9ec* _sqlite3_next_stmt
0001:0000ba28* _sqlite3_stmt_status
0001:0000ba82* _sqlite3_blob_bytes
0001:0000c5ea  _sqlite3_set_authorizer
0001:0000d601* _sqlite3_enable_load_extension
0001:0000d8fd* _sqlite3_free_table
0001:0000e9f0  _sqlite3_complete
0001:0000f2d3  _sqlite3_libversion
0001:0000f31d* _sqlite3_sourceid
0001:0000f327* _sqlite3_libversion_number
0001:0000f331* _sqlite3_threadsafe
0001:0000f4a5* _sqlite3_db_mutex
0001:0000f562  _sqlite3_last_insert_rowid
0001:0000f570  _sqlite3_changes
0001:0000f57b  _sqlite3_total_changes
0001:0000f653* _sqlite3_busy_handler
0001:0000f697  _sqlite3_progress_handler
0001:0000f705  _sqlite3_busy_timeout
0001:0000f74f  _sqlite3_interrupt
0001:0000f761* _sqlite3_trace
0001:0000f7a3* _sqlite3_profile
0001:0000f7e5* _sqlite3_commit_hook
0001:0000f827* _sqlite3_update_hook
0001:0000f869* _sqlite3_rollback_hook
0001:0000f8ab  _sqlite3_errcode
0001:0000f8f1* _sqlite3_extended_errcode
0001:0000f938* _sqlite3_limit
0001:0000f970* _sqlite3_collation_needed
0001:0000f9b4* _sqlite3_collation_needed16
0001:0000f9f8* _sqlite3_global_recover
0001:0000f9ff  _sqlite3_get_autocommit
0001:0000fa0b* _sqlite3_thread_cleanup
0001:0000fa10* _sqlite3_extended_result_codes
0001:000111d8* _sqlite3_db_config
0001:00011204* _sqlite3_config
0001:000170fe* _sqlite3_snprintf
0001:00027681  _sqlite3_value_text
0001:0002766d* _sqlite3_value_text16
0001:0006e71d* _sqlite3_version
0001:0001bde6* _sqlite3_file_control
0001:0001c7de* _sqlite3_bind_parameter_index
0001:0001ce4e* _sqlite3_os_end
0001:0001ce8e* _os2CurrentTime
0001:0001d9be* _sqlite3_os_init
0001:000232e0* _sqlite3_vfs_register
0001:0001d9e1* _sqlite3_initialize
0001:0002129e* _sqlite3_malloc
0001:0001de60* _sqlite3_reset_auto_extension
0001:0001deb0* _sqlite3_shutdown
0001:0001df62* _sqlite3_vmprintf
0001:0001dfd0* _sqlite3_mprintf
0001:0001e213* _sqlite3_realloc
0001:0001f8c6* _sqlite3_set_auxdata
0001:000211f3* _sqlite3_auto_extension
0001:00023216* _sqlite3_soft_heap_limit
0001:00023273* _sqlite3_mutex_alloc
0001:0002338f* _sqlite3_vfs_find
0001:000233fe* _sqlite3_sleep
0001:0002344e* _sqlite3_randomness
0001:000235c0* _sqlite3_test_control
0001:00027645* _sqlite3_value_text16le
0001:00027659* _sqlite3_value_text16be
0001:000276db  _sqlite3_errmsg
0001:00027773  _sqlite3_value_blob
0001:000277b0* _sqlite3_value_bytes16
0001:000277f5  _sqlite3_value_bytes
0001:000278a6  _sqlite3_value_double
0001:0002870f* _sqlite3_value_numeric_type
0001:00028817  _sqlite3_value_int64
0001:00028826* _sqlite3_value_int
0001:00029cc3  _sqlite3_result_int64
0001:00029d10* _sqlite3_result_int
0001:00029e54  _sqlite3_transfer_bindings
0001:00029e9f* _sqlite3_result_zeroblob
0001:00029f53* _sqlite3_clear_bindings
0001:0002af39* _sqlite3_result_value
0001:0002b009  _sqlite3_aggregate_context
0001:0002b898* _sqlite3_create_collation_v2
0001:0002b8f7  _sqlite3_create_collation
0001:0002ba77* _sqlite3_create_module_v2
0001:0002ba98* _sqlite3_create_module
0001:0002bb44* _sqlite3_load_extension
0001:0002c047* _sqlite3_overload_function
0001:0002c0ff  _sqlite3_create_function
0001:0002c1e6  _sqlite3_column_type
0001:0002c209* _sqlite3_column_value
0001:0002c23d* _sqlite3_column_text16
0001:0002c26c  _sqlite3_column_text
0001:0002c29b  _sqlite3_column_blob
0001:0002c2ca* _sqlite3_column_bytes16
0001:0002c2f9  _sqlite3_column_bytes
0001:0002c465  _sqlite3_column_double
0001:0002c491  _sqlite3_column_int64
0001:0002c50a* _sqlite3_column_int
0001:0002c63f  _sqlite3_bind_null
0001:0002c670  _sqlite3_bind_int64
0001:0002c6d5* _sqlite3_bind_int
0001:0002c6fb* _sqlite3_bind_zeroblob
0001:0002cad5* _sqlite3_result_error_toobig
0001:0002cb51* _sqlite3_result_error_code
0001:0002cbdd* _sqlite3_result_text16le
0001:0002cbfc* _sqlite3_result_text16be
0001:0002cc1b* _sqlite3_result_text16
0001:0002cc3d  _sqlite3_result_text
0001:0002d539  _sqlite3_result_blob
0001:0002d91b* _sqlite3_result_error16
0001:0002d948  _sqlite3_result_error
0001:0002e08d* _sqlite3_create_collation16
0001:0002e115* _sqlite3_create_function16
0001:0002e19b* _sqlite3_errmsg16
0001:000304d5* _sqlite3_bind_text16
0001:00030502  _sqlite3_bind_text
0001:0003052f  _sqlite3_bind_blob
0001:000305b4  _sqlite3_bind_double
0001:00030604* _sqlite3_bind_value
0001:000306e7  _sqlite3_result_double
0001:0003090d* _sqlite3_result_error_nomem
0001:00031b12  _sqlite3_result_null
0001:00031d93  _sqlite3_close
0001:0003232e* _sqlite3_backup_finish
0001:000350c5* _sqlite3_backup_step
0001:00038fb8* _sqlite3_blob_write
0001:00038fda* _sqlite3_blob_read
0001:00038ffc  _sqlite3_finalize
0001:000391bb* _sqlite3_blob_close
0001:00039209  _sqlite3_reset
0001:000392d4* _sqlite3_complete16
0001:0003950c* _convertCpPathToUtf8
0001:0003b0ad* _sqlite3_open16
0001:0003b150* _sqlite3_open_v2
0001:0003b16b  _sqlite3_open
0001:0003b774* _sqlite3_backup_init
0001:0004cdfb* _sqlite3_declare_vtab
0001:0004efe3* _sqlite3_prepare16_v2
0001:0004f010* _sqlite3_prepare16
0001:0004f03d* _sqlite3_prepare_v2
0001:0004f1f1  _sqlite3_prepare
0001:0004f276  _sqlite3_step
0001:0005452f* _sqlite3_exec
0001:00061c23* _sqlite3_get_table
0001:00065430* _sqlite3_blob_open
0002:00001ab0* _sqlite3_temp_directory
Module: U:\usr\local446\lib\gcc\i386-pc-os2-emx\4.4.6\libgcc.lib(emx-ctordtor.obj)
0001:00072ee0  ___ctordtorTerm
0001:00072f12  ___ctordtorInit
Module: U:\usr\local446\lib\gcc\i386-pc-os2-emx\4.4.6\libgcc.lib(_divdi3.obj)
0001:00072f50  ___divdi3
Module: U:\usr\local446\lib\gcc\i386-pc-os2-emx\4.4.6\libgcc.lib(_moddi3.obj)
0001:00073090  ___moddi3
Module: U:\usr\local446\lib\gcc\i386-pc-os2-emx\4.4.6\libgcc.lib(_umoddi3.obj)
0001:00073250  ___umoddi3
Module: U:\usr\local446\lib\gcc\i386-pc-os2-emx\4.4.6\libgcc.lib(_udivdi3.obj)
0001:00073370  ___udivdi3
Module: U:\usr\local446\lib\gcc\i386-pc-os2-emx\4.4.6\libgcc.lib(_fixunsdfdi.obj)
0001:00073480  ___fixunsdfdi
Module: U:\tmp\ldconv_libgcc_so_d_a_de0c4f0802a11ec540.lib(emx-eh.obj)
0001:00073525  ___ehInit
0001:000734f0* ___ehTerm


                        +----------------------+
                        |   Imported Symbols   |
                        +----------------------+

Symbol                              Module
======                              ======

___libc_ForkRegisterModule          libc064
___init_dll                         libc064
___libc_Back_termDll                libc064
___libc_ForkDeregisterModule        libc064
__atfork_callback                   libc064
_PyType_GenericNew                  python27
_PyType_Ready                       python27
___stdoutp                          libc064
_PyObject_Print                     python27
__Py_NoneStruct                     python27
_Py_BuildValue                      python27
_PyString_FromString                python27
_PyString_Format                    python27
_PyDict_GetItem                     python27
_PyDict_Size                        python27
_PyDict_DelItem                     python27
_PyObject_CallFunction              python27
_PyDict_SetItem                     python27
_PyArg_ParseTuple                   python27
_PyDict_New                         python27
_PyObject_CallMethod                python27
__Py_ZeroStruct                     python27
_PyErr_SetString                    python27
_PyGILState_Ensure                  python27
_PyErr_Occurred                     python27
_PyGILState_Release                 python27
_PyString_FromStringAndSize         python27
_PyObject_CallFunctionObjArgs       python27
_PyInt_AsLong                       python27
_PyErr_Print                        python27
_PyErr_Clear                        python27
_PyObject_IsTrue                    python27
_PyObject_GetAttrString             python27
_PyObject_CallObject                python27
_PyWeakref_NewRef                   python27
_PyList_Append                      python27
_PyThread_get_thread_ident          python27
_PyErr_Format                       python27
_PyArg_ParseTupleAndKeywords        python27
_PyList_New                         python27
_PyList_GetItem                     python27
_PyWeakref_GetObject                python27
_PyList_Size                        python27
_PyTuple_New                        python27
_PyTuple_SetItem                    python27
_PyBuffer_New                       python27
_PyObject_AsWriteBuffer             python27
_PyUnicodeUCS2_DecodeUTF8           python27
_PyFloat_FromDouble                 python27
_PyInt_FromLong                     python27
_PyFloat_Type                       python27
_PyType_IsSubtype                   python27
_PyBuffer_Type                      python27
_PyUnicodeUCS2_AsUTF8String         python27
_PyString_AsString                  python27
_PyFloat_AsDouble                   python27
_PyObject_AsCharBuffer              python27
_PyExc_ValueError                   python27
_PyEval_SaveThread                  python27
_PyEval_RestoreThread               python27
_PyMem_Free                         python27
_PyImport_ImportModule              python27
_PyModule_GetDict                   python27
_PyDict_GetItemString               python27
_PyString_Concat                    python27
_PyMem_Malloc                       python27
_PyUnicode_Type                     python27
_PyObject_Str                       python27
__PyObject_New                      python27
_PyString_Type                      python27
_PyCallable_Check                   python27
_PyExc_TypeError                    python27
_PyObject_ClearWeakRefs             python27
_PyLong_FromLongLong                python27
_PyOS_snprintf                      python27
__PyObject_NextNotImplemented       python27
_PyIter_Next                        python27
_PyObject_GetIter                   python27
___libc_GLocaleCtype                libc064
_PyObject_HasAttrString             python27
_PyErr_ExceptionMatches             python27
_PyDict_SetItemString               python27
_PyInt_Type                         python27
_PyLong_Type                        python27
__Py_TrueStruct                     python27
_PyObject_Call                      python27
_Py_InitModule4                     python27
_PyModule_AddObject                 python27
_PyExc_StandardError                python27
_PyErr_NewException                 python27
_PyCell_Type                        python27
_PyEval_InitThreads                 python27
_PyExc_ImportError                  python27
_PyType_Type                        python27
_PyTuple_Type                       python27
__Py_NotImplementedStruct           python27
_PyObject_RichCompare               python27
_PyObject_Hash                      python27
_PyTuple_Size                       python27
_PySlice_Type                       python27
_PyExc_IndexError                   python27
_PyTuple_GetItem                    python27
_PyLong_AsLong                      python27
_PyObject_IsInstance                python27
_PyLong_AsLongLong                  python27
_PyList_Type                        python27
_PyDict_Type                        python27
_PyMapping_GetItemString            python27
_PySequence_Check                   python27
_PySequence_Size                    python27
_PySequence_GetItem                 python27
_PyErr_NoMemory                     python27
__CRT_init                          libc064
__CRT_term                          libc064
DosQueryMutexSem                    doscalls
DosReleaseMutexSem                  doscalls
DosRequestMutexSem                  doscalls
DosCloseMutexSem                    doscalls
DosCreateMutexSem                   doscalls
DosGetInfoBlocks                    doscalls
DosSleep                            doscalls
UniFreeUconvObject                  uconv
DosGetDateTime                      doscalls
DosQuerySysInfo                     doscalls
DosFreeModule                       doscalls
DosQueryProcAddr                    doscalls
DosSetFileLocks                     doscalls
DosQueryFileInfo                    doscalls
DosResetBuffer                      doscalls
DosSetFileSize                      doscalls
DosSetFilePtr                       doscalls
DosWrite                            doscalls
DosRead                             doscalls
DosClose                            doscalls
DosForceDelete                      doscalls
UniCreateUconvObject                uconv
UniStrToUcs                         uconv
UniStrFromUcs                       uconv
DosLoadModule                       doscalls
DosQueryPathInfo                    doscalls
DosDelete                           doscalls
DosOpen                             doscalls
DosScanEnv                          doscalls
DosQueryCurrentDisk                 doscalls
__std_memcpy                        libc064
__std_strcpy                        libc064
___ctordtorTerm1                    libc064
___ctordtorInit1                    libc064
__std_memset                        libc064
__std_strcmp                        libc064
__std_strncmp                       libc064
__std_realloc                       libc064
__std_free                          libc064
__std_malloc                        libc064
__std_localtime_r                   libc064
__std_atoi                          libc064
__std_strncat                       libc064
__std_memmove                       libc064
__std_memcmp                        libc064
__std_calloc                        libc064
__std_sprintf                       libc064
__std_qsort                         libc064
___deregister_frame                 gcc446
___register_frame_table             gcc446


                        +--------------------+
                        |   Libraries Used   |
                        +--------------------+

U:\extras\lib\sqlite3.lib
U:\tmp\ldconv_python2_7_dll_a_de0c4f0802a11ec540.lib
U:\usr\local446\lib\gcc\i386-pc-os2-emx\4.4.6\libgcc.lib
U:\tmp\ldconv_libgcc_so_d_a_de0c4f0802a11ec540.lib
U:\usr\lib\libc_alias.lib
U:\usr\local446\lib\libc_dll.lib
U:\usr\lib\libos2.lib
U:\usr\lib\libend.lib


                        +-----------------------+
                        |   Linker Statistics   |
                        +-----------------------+

Stack size:  0000 (0.)
Memory size:  00075550 (480592.)
Link time: 00:00.07
